:020000020000FC
:1000000060C05FC05EC05DC05CC05BC05AC0BFC0A6
:1000100000E829D0089500EC26D0089508950F93A4
:1000200005E40A95F1F70F9108950F930BE01FEF88
:100030001A95F1F70A95D9F70F9108951F930F9329
:10004000007F086008F0046008BBE8DF0F91C398E8
:100050000295007F086008F0046008BBDFDFC398EA
:10006000DEDF1F9108950894E9CF8894E7CF02E37B
:10007000DCDF0A95E9F708E308BBD0DFC398D5DFDA
:10008000D4DF08E308BBD1DF08E308BBC7DFCDDF5F
:1000900008E2E9DF08E2E7DF08E0E5DF01E0E3DFAF
:1000A000C4DF06E0E0DF0EE0DEDFBFDF08954C4492
:1000B000436275746F6E73303430393034432000CE
:1000C00000000FED0DBF03E008BB0CEF07BB0FEF07
:1000D00002BB00E050E000E0102E48D0C8DF09E18C
:1000E00009B9539A549A23D096DFBB27DD27FF27FF
:1000F000C0E6E0E6579A789456D0CE17B9F06191F1
:10010000E13A09F4E0E66F3152F46D3021F4A1EAEE
:1001100000E0102E80DF6A3009F4516007C050FD06
:1001200011D0A23B19F06D93062F9FDFE5CF70DF52
:10013000F0E0EEEAC895002021F0002D96DF319620
:10014000F9CF08957F9367DF70E100E28EDF7A9543
:10015000E1F75EDFA1EA00E0102E0D9186DFA23B01
:10016000E1F704D0507057DF7F910895A1EA00E0D5
:10017000102E00E20D93A23BE9F7A1EA08955F9BE0
:10018000FECF4CB108955D9BFECF3CB908950F930F
:100190000FB70F93F4DF4993C13A09F4C0E60F910A
:1001A0000FBF0F911895839B03C0829B07C00895D2
:1001B0003DE00AD0839BFECF0AD0089532E504D0FB
:1001C000829BFECF04D00895DEDF01D00895002782
:0C01D00033273A95F1F70A95D9F7089506
:00000001FF
